:020000040000FA
:1000000000A804000000000076A9000076A9000006
:1000100076A9000076A9000076A9000076A9000064
:1000200076A9000076A9000076A9000076A9000054
:1000300076A9000076A9000076A9000076A9000044
:1000400076A9000076A9000076A9000076A9000034
:1000500076A9000076A9000076A9000076A9000024
:1000600076A9000076A9000076A9000076A9000014
:1000700076A9000076A9000076A9000076A9000004
:1000800076A9000076A9000076A9000076A90000F4
:1000900076A9000076A9000076A9000076A90000E4
:1000A00076A9000076A9000076A9000076A90000D4
:1000B00076A9000076A9000076A9000076A90000C4
:1000C00076A9000076A9000076A9000076A90000B4
:1000D00076A9000076A9000076A9000076A90000A4
:1000E00076A9000076A9000076A9000076A9000094
:1000F00076A9000076A9000076A9000076A9000084
:1001000076A9000076A9000076A9000076A9000073
:1001100076A9000076A9000076A9000076A9000063
:1001200076A9000076A9000076A9000076A9000053
:1001300076A9000076A9000076A9000076A9000043
:1001400076A9000076A9000076A9000076A9000033
:1001500076A9000076A9000076A9000076A9000023
:1001600076A9000076A9000076A9000076A9000013
:1001700076A9000076A9000076A9000076A9000003
:1001800076A9000076A9000076A9000076A90000F3
:1001900076A9000076A9000076A9000076A90000E3
:1001A00076A9000076A9000076A9000076A90000D3
:1001B00076A9000076A9000076A9000076A90000C3
:1001C00076A9000076A9000076A9000076A90000B3
:1001D00076A9000076A9000076A9000076A90000A3
:1001E00076A9000076A9000076A9000076A9000093
:1001F00076A9000076A9000076A9000076A9000083
:10020000FFFFFF00FFFFFF0076A9000076A90000B6
:1002100076A9000076A9000076A9000076A9000062
:1002200076A9000076A9000076A9000076A9000052
:1002300076A9000076A9000076A9000076A9000042
:1002400076A9000076A9000076A9000076A9000032
:020000040001F9
:104FF000FFFFFF00FFFFFF000000FF000000FF00B9
:105000002F8C20004227A9004507A90042A7AE0027
:10501000FEFF3700F0FF2F0060198800CC22A900A6
:10502000C822A80068A0A800CC02A900C802A90054
:105030000000000000000000CA22AF00A0003700FE
:105040000004EB002635800017368000A406A80077
:10505000A426A800A446A900A466A900A486A900C5
:10506000C206A800C226A800C246A900C266A900BE
:10507000C286A900CC82A800C882A9008000EB00EB
:1050800020022000401188002062A80021E2A80030
:105090002342A80071000700100CB1000900320083
:1050A0002004200020118800C00420002011880066
:1050B0004003200020118800B00220002011880049
:1050C00073003700400D20002011880010002000E0
:1050D000201188002000200020118800B00420004A
:1050E000201188000007EB005C0007009001880099
:1050F0005A00070003E1B7005800070002E1B700BB
:105100000281BF008002780000027800530007008F
:10511000800678005100070080017800028020009E
:105120004E000700005978008301E900FCFF3A00B7
:105130000E04E00003003200E0042000201188008B
:10514000E8FF3700037C2A000328E10010003E003E
:105150000500E00012003A000280200040C0B300C9
:105160000059780000C0B3000059780080CAB3002D
:105170000059780000C0B3000059780000C0B300A7
:105180000059780000C0B3000059780004003700CF
:105190008000EB000005200020118800D1FF3700BF
:1051A000028020000D10A70002003700F1FF2F0041
:1051B000CAFF37000100A60004003700850ABB00C3
:1051C000200424001A0007008000EB0003042000E4
:1051D000B2CABB00B25ABB00B25ABB008301E9009D
:1051E000FBFF3A0010002400110007000304200018
:1051F0000280200014C0BA003204E10009003A0025
:105200003440BA003204E10006003A003440BA00EB
:105210003204E10003003A008301E900F5FF3A009F
:10522000AEFF37006005200020118800ADFF370079
:10523000003B880050052000303B8800A00A200079
:10524000303B880061E7A80000000000000000007B
:1052500061E7AF00FEFF3700000006001A012000E2
:105260008005EB000060FE002202AE000300370064
:105270003011800000074700000006008B05E900A0
:10528000F8FF3A000A05E900F5FF3A002F8C2000EC
:105290000800A600CA22AE006AFF37008560A90098
:1052A0008580A9002342A90021E2A9000221EF0084
:1052B000CC82A900C882A80026358800173688004D
:1052C00068A0A900C802A80000002000601988009A
:1052D00049FF3700F8FF2F005AFF37000008000091
:1052E000C200000000000000000000000000FE00FE
:1052F000FFFFFF00FFFFFF00FFFFFF00FFFFFF00BA
:10530000FFFFFF00FFFFFF00FFFFFF00FFFFFF00A9
:10531000FFFFFF00FFFFFF00FFFFFF00FFFFFF0099
:10532000FFFFFF00FFFFFF00FFFFFF00FFFFFF0089
:0857F000B8FE370004040000BC
:0857F800DFF900007F3F000013
:00000001FF
